:020000020000FC
:1000000019C018951895189518951895189518955C
:100010001895189518951895189518951895189578
:100020000BD51895ECD41895189518951895189522
:100030001895189504E00EBF0FEF0DBF00E004B94E
:100040000FEF05B90FEF07B90FEF08B90EEB0AB9BB
:100050000EEB0BB900E040984198429A5F9808EA8D
:100060001127EE27F1E011930A95E9F780E090E07F
:10007000FDD40535B9F005E5EED4019605E5EBD4E0
:10008000019600E0E8D401960EE0E5D4019607E37E
:10009000E2D4019600E3DFD4019600E0DCD40196BF
:1000A00001E0D9D482E090E0E1D40770000FE8E2EB
:1000B000FCE01127E00FF11F05910093C4000491AB
:1000C0000093C50008E90093C10083E090E0CED41E
:1000D0000093C2005F98FF24EE24DD2470E2672EB7
:1000E00070E000E006BD00E004BD05E005BD01E0F4
:1000F00005BB01E000936E008824789400E0902E08
:10010000F8D0C8E2D1E038E200E209933A95E9F785
:1001100038E200E009933A95E9F708E3EED30CE002
:10012000ECD301E0EAD3E8E0FCE020E034E018D4CE
:100130008BD2E8E8FCE058D082E090E097D40770DA
:10014000000F000F000FEAEBFCE010E0E00FF11FE2
:100150004BD087E090E08AD407700A95000F000F1B
:10016000000FEAEFFCE010E0E00FF11F3DD085D476
:100170006BD2E6EAFCE038D084E090E077D420E06F
:100180000F70022B0F70C02E000F000F000FEAE25D
:10019000FDE010E0E00FF11F27D004E1602FE2EB5B
:1001A000FCE022D085E090E061D40F70000F000FDA
:1001B000000FEAE6FDE010E0E00FF11F15D05DD47E
:1001C00043D2F8D3403270F00C2D0F70043011F48C
:1001D00019D1F7CF9920A9F7C7FE02C01AD2F1CFE3
:1001E0000CD2EFCF0CD0EDCF0591002339F0402F8A
:1001F000EF93FF9302D2FF91EF91F6CF0895423033
:1002000049F00C2D0F70063009F4C1C0013009F41B
:1002100068C17CC0CFD3453009F00895CBD34234B8
:1002200081F04335C1F0433411F1473079F14C345A
:10023000B9F14434C1F1403519F04A34B9F10895A7
:1002400041C0B8D3242FB6D3433079F5022F82E0D2
:1002500090E001D4EFCEAED3242FACD3433029F5B8
:10026000022F85E090E0F7D344D0E4CE0895A2D3E6
:10027000202FA0D34330C9F4022F84E090E0EBD3C9
:100280002C2D207F0F70022BC02ED4CE93D392D36F
:10029000433059F480E090E000E0DDD3F894CACE1A
:1002A00089D388D3089586D385D3089583D34233E1
:1002B000E1F780D34330C9F781E090E000E0CBD391
:1002C000F894B8CA77D3202F75D3433071F7022F33
:1002D000077087E090E0BFD3022F07700A95E8E32C
:1002E000FCE01127E00FF11F049183E090E0B3D30D
:1002F000A1CE85E090E0BAD30F70000FEEE3FCE0F2
:100300001127E00FF11FA590B49008954A30A1F095
:10031000483069F0493061F04B3079F04C3049F0A9
:100320004D3041F0483139F04B3171F0DAC098C1AD
:10033000CAC18AC1A8C1FDC1ABC184C12FC229C233
:1003400026C23EC233C232C235D34B3529F04135C5
:10035000A9F04C36D9F008952DD3443441F34334F9
:1003600039F3413459F3423439F3483431F34C34DE
:1003700009F3423521F34B3419F308951BD341346B
:1003800001F34234F9F24434F1F208952CC14A30B9
:1003900009F14830C9F04930C1F04F31E1F04E3138
:1003A000A9F04D30A1F04031C9F04131C9F04231DE
:1003B000D1F0483171F0493159F04430B9F04C3145
:1003C000B9F04D31C1F0089550C17DC13DC15BC14F
:1003D000CCC189C15DC1E894C7F836C1EBD27EC1FA
:1003E000E894C7F808956894C7F80895E3D208958B
:1003F00001E0802E0895882408950895DBD24D30C1
:10040000E9F708954132C9F7D5D24332B1F7D2D2D4
:10041000413369F0423349F1443349F0453371F3D4
:10042000463329F0483351F34933E9F1089560E048
:10043000C1D24D3071F0A0E0B1E01127A60FB11F7D
:100440004C9363956431A4F3B5D24D30E9F7C2D132
:100450000895A0E0B1E01127A60FB11F00E20C93B0
:1004600063956431B4F3B6D1089564E1A3D24D30FD
:1004700071F0A0E0B1E01127A60FB11F4C93639576
:100480006832A4F397D24D30E9F7A4D10895A0E0E3
:10049000B1E01127A60FB11F00E20C9363956832FB
:1004A000B4F398D1089560E085D24D3071F0A0E0AA
:1004B000B1E01127A60FB11F4C9363956832A4F3E6
:1004C00079D24D30E9F786D10895A0E0B1E0112747
:1004D000A60FB11F00E20C9363956832B4F37AD192
:1004E0000895992041F04B3109F0089563D24D33BE
:1004F00009F0089562C04A30B1F0483079F04930CF
:1005000071F04B3089F04C3059F04D3051F048319A
:1005100049F04B31B1F04F3111F10895A1C0D3C072
:1005200093C0B1C006C1B4C08DC05AC052C031C161
:100530002EC146C13BC13AC153CF55CF2FC153C085
:1005400026C138D2403489F34437A9F14D33A9F19B
:10055000423561F3473579F10F910F9141CE2AD29F
:10056000413051F3423049F34A3041F34D30C9F242
:10057000443229F3423421F34334E9F04534D9F0CD
:10058000403499F2089516D2443441F2433439F29A
:10059000423449F2483441F24C3419F2423539F2CE
:1005A0004B3431F2089506D2413419F2423411F23B
:1005B000443409F20895FED10895FCD1413319F075
:1005C000423321F0089501E0902E089500E0902E2E
:1005D0000895F0D1042F85E090E03DD28ADE0895A1
:1005E000E894C7F831C0E6D1242F2A95E3D14230F0
:1005F00011F404E1200F422F71C0A0E0B1E01127F7
:10060000A60FB11F4C930ED16395683209F460E0D8
:100610000895A0E0B1E01127A60FB11F4C93639598
:10062000683211F0D7D00895A0E0B1E0C4E1D1E084
:1006300014E108810D9300E209931A95D1F764E162
:10064000C9D008956627089500E260E0A0E0B1E017
:100650000D9363956832E1F760E08824BBD008957C
:10066000662309F468E26A950895662311F467E247
:1006700001C06A95A0E0B1E01127A60FB11F00E20A
:100680000C93A8D00895643164E10CF460E00895FF
:10069000C7FC08C0643118F004E1601B089504E150
:1006A000600F089564311CF404E1600F0895A0E028
:1006B000B1E0C4E1D1E014E108810D9300E20993B7
:1006C0001A95D1F787C0C7FC05C06395683209F455
:1006D00060E0089563956832E1F7A6CF8824483238
:1006E0000CF4642F0895643194F4633109F408958F
:1006F0006F936395A0E0B1E01127A60FB11F00E250
:100700000D9363956431D9F765D06F910895683280
:1007100009F408956F936395A0E0B1E01127A60F47
:10072000B11F00E20D9363956832D9F753D06F91F2
:100730000895643160E068F064E1A0E0B1E0112761
:10074000A60FB11F00E20D9363956832D9F764E1FB
:1007500041C0A0E0B1E01127A60FB11F00E20D9348
:1007600063956431D9F760E035C0673208F00895C9
:100770006F936395A0E0B1E01127A60FB11F00E2CF
:100780000D9363956832D9F725D06F91089567E28C
:100790000895643163E108F067E20895643118F068
:1007A00004E1601B089504E1600F089564E1C1DF76
:1007B000603029F0FFD04D3011F01FDFF9CF0895E0
:1007C00060E0B7DF643129F0F5D04D3011F015DF6E
:1007D000F9CF08958824A0E0B1E0C8E2D1E030E08C
:1007E0000D911881011739F008830F9300E8030F6A
:1007F00084D00F916BD009913395343189F7A4E1FE
:10080000B1E030E00D911881011739F008830F93A2
:1008100000EC030F72D00F9159D009913395343108
:1008200089F70895CA2FDB2F0C9108A700E510E087
:10083000C00FD11F00E080FC01E00883643124F484
:1008400000E8060F5AD005C008EA162F1451010F10
:1008500054D00C913BD00895C8E2D1E030E008A517
:10086000002329F000E8030F48D008812FD0099118
:1008700033953431A1F730E008A5002329F008EAC8
:10088000030F3BD0088122D0099133953431A1F771
:100890000895C8E2D1E030E008A5002329F000E87F
:1008A000030F2BD000E212D0099133953431A1F718
:1008B00030E008A5002329F008EA030F1ED000E26B
:1008C00005D0099133953431A1F70895EA2DFB2D18
:1008D0001591112339F0011711F01591F9CF0491F9
:1008E0000AD00895EEE8FAE015911123C9F3011733
:1008F000B1F31591F9CF2ED002C02CD04298419877
:10090000102F037C17951F7D11FD10621C73012BA6
:100910001FEF05B914B9409A000000004098429AB0
:100920000FEF05B900E004B9089514D001C0429852
:10093000419A409A0000000003B14098429A102F5B
:10094000037C111F1B7F16FD14601C73012B409844
:10095000429A08950F93EBDF07FDFDCF0F910895A5
:10096000330F330F330F220F220F26952064022FEF
:10097000C4DF0591C0DF23953A95C9F708953490F7
:10098000332021F0532D0DD03196F9CF08950F70FB
:100990000A3018F40063502F04C009500064502F2F
:1009A00000C05E99FECF0091C00005FFFACF5093C2
:1009B000C6000895789400000000F894772339F079
:1009C000723019F466DF70E002C046DF70E0DD20AF
:1009D00089F3EF93FF93E8ECF1E00027EF0DF01FB0
:1009E0000081DA94F39410E8F11609F4FF241D2D28
:1009F0000E3608F45F98402FFF91EF9118952FB6AF
:100A0000EF93FF930F93E8ECF1E00027EE0DF01F5A
:100A10000091C60000830E2D0395003809F40027CD
:100A2000E02ED3940D2D003710F05F9A00380F910F
:100A3000FF91EF912FBE18952FB60F936A9429F06E
:100A4000062D003129F472E003C070E2672E71E0D8
:100A50000F912FBE1895F999FECF2FB6F89492BD3D
:100A600081BD00BDFA9AF99A2FBE0895F999FECF7B
:100A700092BD81BDF89A00B5089520EA10E000E02B
:100A80000A95F1F71A95E1F72A95D1F708957F2095
:100A90009BAF9CA59DAE9EB79FA8A49BA59CA69D21
:100AA000A79EA89FA920AA20ABB5ACB6ADA9AEBBA6
:100AB000AFBCB020B120B220B320B420B520B68F97
:100AC000B720B820B920BA20BB20BC20BDA4BEA648
:100AD000BF20C020C120C220C320C420C520C6AB77
:100AE000C7AAC820C920CA20CB20CC20CDDFCE2069
:100AF000CF03D020D120D220D320D420D500D6209F
:100B0000D720D820D920DA20DB20DC20DD20DE2011
:100B1000DF20E020E1E0E220E320E4ADE5ACE6EA1E
:100B2000E720E820E920EA20EB20EC20ED20EEBFD2
:100B3000EFB4F0BFF1B4F22DF320F420F5D3F6B802
:100B4000F720F820F9B2FAB1FBCDFC20FD1FFE2002
:100B5000FF20000023A5D500000040855B015C80DC
:100B60005DD27B827C977D8A7E02D500000040D2D8
:100B70005B8E5C995D9A7B847C947D817EE0D50060
:100B800000005B925CAE5D8F7B917CAF7D83D50076
:100B90000000240340905B8E5C995D8F5E9A6082BA
:100BA0007B847C947D837E81D50000005B015D8227
:100BB00060977B857C957D8A7EA9D500000023A760
:100BC0005BA95C9C5D9F7BB17C9BD50000005CA613
:100BD000D5000000240340905B925CAE5D8F5E9A6E
:100BE00060827B917CAF7D837E81D5000000409048
:100BF0005B925CAE5D9E5E9A60827B917CAF7D83F2
:100C00007E81D5000000000006091C081C090600B2
:100C10000E0A0E00000000000A00000000000000A4
:100C2000110E1111110E110033006700CF009E014B
:100C30003C0378060C0019000E0C2E2C3E3C060CD2
:100C40005A0B6E0B540B820B920BAC0BBE0BCE0BE4
:100C5000D40BEE0B060C060C060C060C060C303101
:100C6000323334353637383930313233343536373C
:100C70003839303132333435363738383839303125
:100C800032333435363738394A3220363530202041
:100C9000202020205665722E20312E364261756448
:100CA000726174653A00456D756C6174696F6E3A76
:100CB0002000466F6E743A20000020393630300034
:100CC0000000203438303000000020323430300052
:100CD000000020313230300000002020363030005B
:100CE0000000202033303000000033383430300032
:100CF00000003139323030000000204E20382031E1
:100D00000000204E203720310000204520382031BF
:100D100000002045203720310000204F20382031AE
:100D20000000204F2037203100004453503830302D
:100D300020004550534F4E2020004550534F4E2029
:100D400020004550534F4E20200041454445582037
:100D5000200055544320502F5400555443205354E1
:100D600044004344373232302000552E532E412E5A
:100D700020004672656E636820004765726D616E83
:100D80002000552E4B2E2020200044656E2E204939
:100D9000200053776564697368004974616C792039
:100DA00020005370616E697368004A6170616E2043
:100DB00020004E6F72776179200044656E2E49499C
:020DC000200011
:1018000019C0189518951895189518951895189544
:101810001895189518951895189518951895189560
:1018200018951895CCD11895189518951895189560
:101830001895189504E00EBF0FEF0DBF00E004B936
:101840000FEF05B90FEF07B90FEF08B90EEB0AB9A3
:101850000EEB0BB900E040984198429A5F9808EA75
:101860001127EE27F1E011930A95E9F7E0E0F0E0A7
:1018700004910F3F59F080E090E0C9D1053529F47B
:1018800081E090E0C4D1053509F4D4C381E090E053
:10189000019600E0B1D101960EE0AED105B7102F50
:1018A000016005BF12E015BF82E090E0B0D10F3FAC
:1018B00009F400E00770000FECE1FCE11127E00FF4
:1018C000F11F05910093C40004910093C50008E93D
:1018D0000093C10083E090E09AD10F3F09F40EE03D
:1018E0000093C2005F98FF24EE24DD24789408E37F
:1018F000F8D00CE0F6D001E0F4D000C0C6D009D09A
:10190000D2D0E4E5FCE1C4D080E090E00FEF74D1E8
:1019100091C3772450D0C7D0882839F41ED009D07D
:101920007394072D0033B1F7F5CF47B640FCFDCFD8
:101930000895E8E6FCE1ACD0072D029503D0072D11
:1019400001D008950F700A3018F40063402F91C041
:1019500009500064402F8DC00895CF93DF93EF931B
:10196000FF93C8E8D1E080E490E006E0FF27E72D90
:10197000EE0FFF1F0A95E1F733E014D031E112D0EA
:101980000990199031E00ED032960297C9F7E054D1
:10199000F04035E007D031E105D0FF91EF91DF91C4
:1019A000CF91089547B640FCFDCF5FB6F89437BF9E
:1019B000E8955FBE08951FD034E0A8E8B1E023D0D9
:1019C000082D0230E1F30130A9F00A2D003041F476
:1019D0000B2D083129F417D0082D013059F0FBCF19
:1019E00000E1E8E7F1E011911D930A95E1F73A95DE
:1019F00031F708950895A8E8B1E010E40FEF0D93D2
:101A00001A95E9F70895BBD04A33E9F71ED0203084
:101A100049F1922E1AD0B22E18D0A22E16D0822EB4
:101A200002D013D0089510E1EF93FF93E8E7F1E0BF
:101A30000FEF01931A95E9F7E8E7F1E006D021935B
:101A40009A94E1F7FF91EF91089505D0242F229504
:101A500002D0242B089593D04A3310F047530895B1
:101A60004F700895F2DFF1DFF0DFEFDF01E0802E4D
:101A70000895A0E0B1E01127A60FB11F4C931ED02E
:101A80006395683209F460E008950DD0ECE2FCE162
:101A90000591002339F0402FEF93FF93EADFFF9188
:101AA000EF91F6CF089500E260E0A0E0B1E00D9381
:101AB00063956832E1F760E001D00895C0E0D1E0BD
:101AC00000E80FD034E109910AD03A95E1F734E10A
:101AD00000EC07D0099103D03A95E1F708952ED094
:101AE00002C02CD042984198102F037C17951F7D7F
:101AF00011FD10621C73012B1FEF05B914B9409A38
:101B0000000000004098429A0FEF05B900E004B9C8
:101B1000089514D001C04298419A409A00000000F4
:101B200003B14098429A102F037C111F1B7F16FDB2
:101B300014601C73012B4098429A08950F93EBDFB9
:101B400007FDFDCF0F9108953490332021F0532DE0
:101B50000DD03196F9CF08950F700A3018F4006354
:101B6000502F04C009500064502F00C05E99FECF72
:101B70000091C00005FFFACF5093C60008957894F5
:101B800000000000F894DD20D1F30F931F93EF9332
:101B9000FF93E8ECF1E00027EF0DF01F0081DA94ED
:101BA000F39410E8F11609F4FF241D2D0E3608F405
:101BB0005F98402FFF91EF911F910F9118952FB6CD
:101BC000EF93FF930F93E8ECF1E00027EE0DF01F89
:101BD0000091C60000830E2D0395003809F40027FC
:101BE000E02ED3940D2D003710F05F9A00380F913E
:101BF000FF91EF912FBE1895F999FECF2FB6F8946B
:101C000092BD81BD00BDFA9AF99A2FBE0895F99947
:101C1000FECF92BD81BDF89A00B5089533006700EC
:101C2000CF009E013C0378060C00190057616974CF
:101C3000696E6720666F722070726F6772616D20C7
:101C400066696C65206174203936303020626175B8
:101C5000642E0000466C6173682055706461746581
:101C600020646F6E652E00005772697465205061A4
:101C700067652000436F7079726967687420286314
:101C800029203230303820432E204E6F726D616E25
:101C90002043616D7062656C6C20616C6C207269B0
:0E1CA000676874207265736572766564000073
:00000001FF
